:100000000C9444050C948C050C948C050C948C0574
:100010000C948C050C948C050C948C050C948C051C
:100020000C948C050C948C050C94010D0C94D30D40
:100030000C94FE1C0C948C050C948C050C948C0573
:100040000C948C050C948C050C948C050C948C05EC
:100050000C948C050C94721D0C948C050C948C05DE
:100060000C948C050C948C050C948C050C948C05CC
:100070000C948C050C948C050C948C050C948C05BC
:100080000C948C050C948C050C948C050C948C05AC
:100090000C948C050C948C050C948C050C948C059C
:1000A0000C948C050C948C050C948C05400E620EFF
:1000B000550F620E550FA70ECA0E550F1F0F320FA8
:1000C000721272129C129C12F7122B1339153915E9
:1000D000421339152D142D14F3143915081526154E
:1000E000507C7E8051634F621B7B35198029102C18
:1000F0007F37808059585A5B1D7A78060E8011052B
:10010000343836805C575D5E070479090D3A0B0A76
:100110007D330F3052808080161439150C3C18172F
:1001200080808080808080808080808080808080CF
:100130002E2D2731532A5455201F8021263B24235E
:100140002F1312285F5660611A1E2B08253D1C22B2
:10015000444342454C4E494B80808080413E403F65
:100160000A4B6579626F6172642073746172742ED8
:100170000A000A55534220636F6E6669677572659F
:10018000642E0A000A0A544D4B3A63323135373136
:1001900033662B2F4C5546410A0A002C0346004378
:1001A000003900380030004300200041006C00742A
:1001B00000200043006F006E00740072006F006C3E
:1001C000006C006500720000000A0354004D004BF3
:1001D000002E0000000403090409028D000501003F
:1001E000A0320904000001030101000921110100EE
:1001F000012240000705810308000A0904010001EB
:1002000003010200092111010001224D00070582AE
:100210000308000A0904020001030000000921117B
:100220000100012236000705830308000A090403C0
:100230000002030000000921110100012222000731
:1002400005840320000107050403200001090404BC
:1002500000010300000009211101000122390007FB
:100260000585032000011201100100000008EDFEC9
:100270000C9800010102000105010906A101050712
:1002800019E029E715002501950875018102050887
:1002900019012905950575019102950175039101D3
:1002A0000507190029F71500250195F87501810248
:1002B000C00631FF0974A1010975150026FF0095DC
:1002C00020750881020976150026FF009520750823
:1002D0009102C005010980A101850216010026379F
:1002E000001A81002AB700751095018100C0050C25
:1002F0000901A1018503160100269C021A01002AAA
:100300009C02751095018100C005010902A1010937
:1003100001A100050919012905150025019505759B
:10032000018102950175038101050109300931152B
:1003300081257F95027508810609381581257F95ED
:100340000175088106050C0A38021581257F950183
:1003500075088106C0C005010906A101050719E05D
:1003600029E7150025019508750181029501750899
:10037000810105081901290595057501910295016D
:10038000750391010507190029FF150026FF009547
:100390000675088100C0636F6E73756D65723A20D3
:1003A000253034580A0073797374656D3A2025300E
:1003B00034580A000A002530325820006B657962F3
:1003C0006F6172643A20004C45443A20253032581F
:1003D0000A00253032583A20253031366225730A1A
:1003E00000722F632030313233343536373839419B
:1003F00042434445460A0064656C5F6B65795F6201
:1004000069743A2063616E27742064656C3A202514
:100410003032580A006164645F6B65795F626974A9
:100420003A2063616E2774206164643A202530327B
:10043000580A004F6E6573686F743A2074696D6571
:100440006F75740A00290A002575002F00257500B4
:100450005D2800256400200025640020002564003C
:1004600020002564007C0025303258006D6F7573C4
:10047000656B6579205B62746E7C782079207620CC
:10048000685D287265702F61636C293A205B006D8E
:100490006B5F776865656C5F74696D655F746F5FCE
:1004A0006D6178203D2025640A006D6B5F7768657B
:1004B000656C5F6D61785F7370656564203D2025B4
:1004C000640A006D6B5F74696D655F746F5F6D6169
:1004D00078203D2025640A006D6B5F6D61785F7345
:1004E00070656564203D2025640A006D6B5F696E50
:1004F00074657276616C203D2025640A006D6B5F27
:1005000064656C6179203D2025640A006D6B5F771E
:100510006865656C5F74696D655F746F5F6D617848
:10052000203D2025640A006D6B5F776865656C5F10
:100530006D61785F7370656564203D2025640A00F5
:100540006D6B5F74696D655F746F5F6D6178203D81
:100550002025640A006D6B5F6D61785F737065655F
:1005600064203D2025640A006D6B5F696E746572BE
:1005700076616C203D2025640A006D6B5F64656CBC
:100580006179203D2025640A000A00257500363A6D
:1005900020776865656C5F74696D655F746F5F6D0A
:1005A00061783A20000A00257500353A20776865A1
:1005B000656C5F6D61785F73706565643A20000AF1
:1005C00000257500343A2074696D655F746F5F6D46
:1005D00061783A20000A00257500333A206D617871
:1005E0005F73706565643A20000A00257500323A31
:1005F00020696E74657276616C286D73293A2000EB
:100600000A00257500313A2064656C6179282A3129
:10061000306D73293A20000A092D2056616C7565EA
:1006200073202D0A004D3E004D25643E20003F0002
:100630007365742064656661756C740A00433E20BE
:100640000077686572652064656C74613A20637533
:1006500072736F723D25642C20776865656C3D254B
:10066000640A53656520687474703A2F2F656E2E86
:1006700077696B6970656469612E6F72672F77693E
:100680006B692F4D6F7573655F6B6579730A000A2F
:10069000092D204D6F7573656B6579202D0A4553C3
:1006A000432F713A09717569740A313A0964656CAE
:1006B0006179282A31306D73290A323A09696E74DA
:1006C000657276616C286D73290A333A096D617819
:1006D0005F73706565640A343A0974696D655F74A7
:1006E0006F5F6D61780A353A09776865656C5F6D93
:1006F00061785F73706565640A363A097768656585
:100700006C5F74696D655F746F5F6D61780A0A7004
:100710003A097072696E742076616C7565730A644B
:100720003A097365742064656661756C74730A7543
:10073000703A092B310A646F776E3A092D310A70CD
:100740006775703A092B31300A7067646F776E3ABB
:10075000092D31300A0A7370656564203D20646597
:100760006C7461202A206D61785F73706565642008
:100770002A2028726570656174202F2074696D6568
:100780005F746F5F6D6178290A003F004D3E200065
:10079000433E20004C25640A000A092D20436F6E59
:1007A000736F6C65202D0A4553432F713A0971759B
:1007B00069740A6D3A096D6F7573656B65790A0026
:1007C0000A092D204D61676963202D0A643A096486
:1007D000656275670A783A096465627567206D61BC
:1007E000747269780A6B3A096465627567206B6593
:1007F00079626F6172640A6D3A0964656275672097
:100800006D6F7573650A763A0976657273696F6EF6
:100810000A733A097374617475730A633A09636FF2
:100820006E736F6C65206D6F64650A302D343A0904
:100830006C61796572302D34284631302D4634296B
:100840000A506175733A09626F6F746C6F61646509
:10085000720A6E3A094E4B524F0A003F004E4B52FD
:100860004F3A206F66660A004E4B524F3A206F6E29
:100870000A0074696D65725F72656164333228299C
:100880003A202530346C580A006B6579626F6172CA
:10089000645F6E6B726F3A2025580A006B6579624F
:1008A0006F6172645F69646C653A2025580A006B59
:1008B0006579626F6172645F70726F746F636F6C81
:1008C0003A2025580A00686F73745F6B6579626F10
:1008D0006172645F6C65647328293A2025580A00A8
:1008E0000A092D20537461747573202D0A00474343
:1008F000433A20352E342E30204156522D4C494259
:10090000433A20322E302E30204156525F4152431E
:10091000483A20617672350A004F5054494F4E5381
:100920003A204C554641204D4F5553454B45592093
:1009300045585452414B455920434F4E534F4C4517
:1009400020434F4D4D414E44204E4B524F204B457E
:10095000594D41505F53454354494F4E203430392F
:10096000360A004255494C443A206332313537311A
:1009700033662B202831343A30363A3435204F63F1
:10098000742020312032303139290A005649443A46
:100990002030784645454428544D4B2E2920504957
:1009A000443A203078393830432846433938304388
:1009B00020416C7420436F6E74726F6C6C65722989
:1009C000205645523A203078303130300A004445C4
:1009D00053433A20544D4B2E206B6579626F617200
:1009E00064206669726D7761726520666F72204659
:1009F00043393830430A000A092D2056657273695D
:100A00006F6E202D0A000A6D6F7573653A206F6650
:100A1000660A000A6D6F7573653A206F6E0A000AE8
:100A20006B6579626F6172643A206F66660A000ACC
:100A30006B6579626F6172643A206F6E0A000A6DAD
:100A400061747269783A206F66660A000A6D617493
:100A50007269783A206F6E0A000A64656275673AB7
:100A6000206F6E0A000A64656275673A206F6666D9
:100A70000A000A0A626F6F746C6F616465722E2ED1
:100A80002E2000433E20000011241FBECFEFDAE0ED
:100A9000DEBFCDBF04B603FE28C08091A4039091B1
:100AA000A503A091A603B091A7038730904BA74060
:100AB000B04BD9F41092A4031092A5031092A60390
:100AC0001092A70314BE0FB6F894A8958091600009
:100AD000886180936000109260000FBE1092010840
:100AE00010920008E0E0F8E3099511E0A0E0B1E021
:100AF000ECEDFBE402C005900D92AE33B107D9F7DF
:100B000023E0AEE3B1E001C01D92A43AB207E1F7E1
:100B10000E94C8090C94EC250C940000FF93EF93FD
:100B2000E0913E01F0913F01309709F00995EF9176
:100B3000FF910895FC018591803011F0EFDFFBCF2C
:100B40000895FF27E0E230E247FF0CC0419597FF90
:100B500009C0EDE26095709580959095611D711DBD
:100B6000811D911D27FF02C0219530E350E2AA2785
:100B7000660F771F881F991FAA1FA41710F0A41BC8
:100B800063955A95A9F7AA3008F0A95FA05DAF93C5
:100B9000F395611571058105910541F7ED3211F469
:100BA000EF93F395F21718F43F93F395FBCF8F91E2
:100BB000B5DFFA95E1F70895E991F99185918030D3
:100BC00021F0853219F0AADFF9CF089520E0E894EA
:100BD00055915532C1F3503311F4689455915A33FD
:100BE00048F4505390F3220F022E220F220F200DB3
:100BF000250FF4CF0EF4219589919991533619F36D
:100C0000533729F1533559F1BC0188279927E894C6
:100C10005C3621F48991999168945591543639F450
:100C200046EF7EF077FF0DC08FEF9FEF0AC055377C
:100C30004AE039F0583540E121F0523642E009F0FF
:100C40000895FF93EF937DDFEF91FF91B7CFFF936F
:100C5000EF93FC0181918030B9F360DFFBCFFF930C
:100C6000EF9368DFF1CFDF93CF93CDB7DEB7259653
:100C7000A3DFCF91DF91089584B18F6084B93E984E
:100C8000469A3F9A8AB1806F8AB95F9A479884B131
:100C9000806784B985B18F7885B9E0E5F1E011927C
:100CA000119281E0E036F807D1F7E0E4F1E080E569
:100CB00091E0119211928E179F07D9F780E591E08C
:100CC000909363018093620180E491E090936101CD
:100CD0008093600108958F929F92BF92CF92DF928E
:100CE000EF92FF920F931F93CF93DF938091600158
:100CF0009091610120916201309163013093610113
:100D0000209360019093630180936201E12CF12CA8
:100D1000C1E0D0E00FEF10E085B1807F8E2985B96A
:100D2000BE010E2C02C0660F771F0A94E2F74B013A
:100D30008094909440E050E08BB1282F2F78CA0126
:100D400034E0880F991F3A95E1F7822B8BB98AE03E
:100D50008A95F1F700C09A01220F331FE0916001DC
:100D6000F0916101E20FF31F808191818623972327
:100D7000892B09F0479AA5E3AA95F1F70000B6B4CC
:100D80005F98BAE0BA95F1F700C0E0916201F09186
:100D900063016F01C20ED31ED601369B06C08D9132
:100DA0009C9111978821992105C08D919C91119753
:100DB000862B972B8D939C9386B5CB2CD12C8B15A2
:100DC00028F086B590E08C199D0906C0B6B4C8011C
:100DD0008C199D098B0D911D069768F0809160011B
:100DE00090916101820F931FDC018D919C91E20F24
:100DF000F31F91838083BAE1BA95F1F700C0479859
:100E00005F9A80EA8A95F1F74F5F5F4F483051054E
:100E100009F092CFA0916201B0916301E09160016D
:100E2000F091610150962D913C9151978089918963
:100E30002817390711F00E943C1DAFEFEA1AFA0A91
:100E4000B0E1EB16F10409F067CF81E0DF91CF91BB
:100E50001F910F91FF90EF90DF90CF90BF909F90E8
:100E60008F9008952091620190916301E22FF92FF4
:100E7000E80FF11DE80FF11D80819181089580FF39
:100E800002C02C9A01C02C9881FF02C02D9A01C08B
:100E90002D9882FF02C02E9A08952E980895809171
:100EA00088020895CF93DF9300D01F92CDB7DEB7AD
:100EB0009C0180919B03843019F593E099833B83D7
:100EC0002A839093E9008FEF9091E800815095FD7F
:100ED00006C095ED9A95F1F700008111F5CF80914C
:100EE000E80085FF0DC040E050E063E070E0CE0117
:100EF00001960E94F50A8091E8008E778093E800C1
:100F00000F900F900F90DF91CF910895CF93DF93C3
:100F100000D01F92CDB7DEB720919B03243031F56E
:100F200022E02983805891099B838A8383E0809300
:100F3000E9008FEF9091E800815095FD06C095ED96
:100F40009A95F1F700008111F5CF8091E80085FFB7
:100F50000DC040E050E063E070E0CE0101960E94D9
:100F6000F50A8091E8008E778093E8000F900F904B
:100F70000F90DF91CF91089520919B032430F1F4DD
:100F800022E02093E9002FEF3091E800215035FD59
:100F900006C035ED3A95F1F700002111F5CF20910B
:100FA000E80025FF0BC040E050E065E070E00E94E3
:100FB000F50A8091E8008E778093E8000895CF933A
:100FC000DF9320919B03243009F04AC0EC0180910B
:100FD0000F018823E1F0809110018823C1F085E0A2
:100FE0008093E90081E8815049F09091E80095FDF7
:100FF00005C09AE29A95F1F700C0F5CF8091E8001C
:1010000085FF2EC040E050E060E270E019C081E052
:101010008093E90081E8815059F09091E80095FDB6
:1010200007C0EFE3F1E03197F1F700C00000F3CF24
:101030008091E80085FF14C040E050E068E070E077
:10104000CE010E94F50A8091E8008E778093E80037
:1010500080E2FE01A8E6B2E001900D928A95E1F7E8
:10106000DF91CF910895CF93C0916601C1110BC05C
:101070000E943C1D643C79408105910520F081E08F
:1010800080936601C1E08C2FCF910895CF93C82F34
:101090000E943308882309F448C00FB607FE45C0F4
:1010A00080919B03843009F040C08091E9008F70EB
:1010B0002091EC00922F917020FD90E8892B94E014
:1010C0009093E9009091EB0090FF2CC09091EE007E
:1010D00097FF28C09091030120910201291709F47C
:1010E00047C02091E80025FF1DC0E0910001F0916C
:1010F0000101E90FF11D30819F5F209104019223CE
:10110000909303013093F1009091E80095FDE2CFB8
:101110009091E80090FFDECF9091E8009E77909349
:10112000E800D8CF8F708093E9008091020190E0B1
:10113000AC014F5F5F4F30910401232F30E0242337
:1011400035234091030150E024173507D1F0209159
:10115000000130910101F901E80FF91FC08380916E
:1011600002018F5F9091040189238093020109C0DD
:101170009091E80095FFD6CFC093F1008F708093D7
:10118000E90080E0CF91089580919A03811109C010
:101190000E94860C0E94E30C8091E20084608093A0
:1011A000E200089510929A0308950895089542E088
:1011B00061EC81E00E94FF0B42E061EC82E00E9462
:1011C000FF0B42E061EC83E00E94FF0B42E261EC26
:1011D00084E00E94FF0B42E261EC85E00C94FF0B7F
:1011E00080919D03833009F455C030F4813071F053
:1011F000823009F48EC008958A3009F47AC08B30A9
:1012000009F460C0893009F09CC020C080919C0323
:10121000813A09F096C08091E800877F8093E800CA
:101220008091A0039091A103892B21F460E288E6CC
:1012300092E003C060E080E090E070E00E94400B2C
:101240008091E8008B778093E800089580919C035B
:10125000813209F076C08091A0039091A10300979C
:1012600019F0049709F06DC08091E800877F8093A2
:10127000E8008091E80082FD05C080919B03811108
:10128000F8CF5FC08091F100809388028091E800E0
:101290008B7753C080919C03813A09F052C08091B2
:1012A000A0039091A103892B09F04BC08091E80025
:1012B000877F8093E8008091E80080FFFCCF8091D9
:1012C0000F0136C080919C038132D9F58091A00333
:1012D0009091A103892BA9F58091E800877F8093E5
:1012E000E8000E94340C80919E0380930F010C94BF
:1012F000221280919C03813221F58091E800877F42
:101300008093E8000E94340C80919F0380938902AF
:10131000089580919C03813AA1F48091E800877F31
:101320008093E8008091E80080FFFCCF80918902E3
:101330008093F1008091E8008E778093E8000C9410
:10134000340C08958091880280936701109288027E
:101350000E94ED100C9422120C94A2090E94BC1C55
:1013600080919903882329F00E94E51C81110C9437
:10137000DF0A08950E94FA1C809167018093880219
:1013800008950C94BA0908950C94C3090C94C309E8
:10139000CF9384B7877F84BF0FB6F894A8958091C8
:1013A0006000886180936000109260000FBE90E042
:1013B00080E80FB6F89480936100909361000FBEAF
:1013C00086E498E00E947C1C85E091E00E946D0F0D
:1013D00084E891E00E949A050E94C6090E942C10A0
:1013E0000E94860C0E94E30C8091E200846080934E
:1013F000E20078940E942E1080919B03843019F0B3
:101400000E94C309F9CF82E791E00E949A050E94E9
:10141000C40980E691E00E949A05C4E080919B0394
:10142000853019F40E94AE09F9CF0E943210209144
:10143000E4003091E50080916401909165012817E6
:10144000390761F38091E4009091E5009093650184
:10145000809364010E943308882301F380919B03E9
:101460008430E1F68091E9008F702091EC00922F9A
:10147000917020FD90E8892BC093E9009091EB00DA
:1014800090FF43C09091EE0097FF3FC09091030101
:1014900020910201291709F12091E80025FF1DC0C4
:1014A000E0910001F0910101E90FF11D30819F5F92
:1014B000209104019223909303013093F1009091C5
:1014C000E80095FDE3CF9091E80090FFDFCF909189
:1014D000E8009E779093E800D9CF9091F300209197
:1014E000F20030E0392B232B81F09091E80090FF3F
:1014F0000CC09091E80095FF03C01092F100F9CF65
:101500009091E8009E779093E8008F708093E900B7
:1015100085CF292F332723303105C9F060F42130DE
:10152000310581F02230310509F041C08DE890E0AD
:1015300029ED31E040C021323105E1F022323105A0
:1015400031F135C082E190E026E632E034C09927DF
:101550008130910549F028F0029749F5EBE9F1E077
:1015600005C0E5EDF1E002C0E9ECF1E0849190E026
:101570009F0121C06530D8F4E62FF0E0EE0FFF1F89
:10158000E85DFE4F2081318189E090E014C0653034
:1015900070F470E0FB01EE0FFF1FE25EFE4F208152
:1015A0003181FB01E75EFE4F808190E004C080E066
:1015B00090E020E030E0FA0131832083089580E15B
:1015C00089BD82E189BD09B400FEFDCF8091D800BC
:1015D0008F7D8093D8008091E00082608093E0004E
:1015E0008091E00081FDFCCF0895CF92DF92EF92D1
:1015F000FF920F931F93CF93DF93EC018B017A013E
:101600000E94530C811133C0E114F10439F0F70149
:1016100080819181081B190BC80FD91FC12CD12CB7
:101620000115110519F18091E80085FD16C0809122
:10163000E8008E778093E800E114F10449F0F701A7
:1016400080819181C80ED91ED182C08285E00FC0F1
:101650000E94530C882321F30AC089918093F100E2
:1016600001501109FFEFCF1ADF0ADACF80E0DF91D6
:10167000CF911F910F91FF90EF90DF90CF90089541
:101680002091A2033091A3032617370748F0611574
:10169000710539F42091E8002E772093E80001C00D
:1016A000B901FC0120E06115710579F180919B037E
:1016B0008823F1F18530F1F18091E80083FD3CC091
:1016C0008091E80082FD2EC08091E80080FFEBCF82
:1016D0002091F3008091F20090E0922B611571054A
:1016E00051F08830910538F421912093F100615038
:1016F00071090196F3CF21E0089709F020E080916D
:10170000E8008E778093E800CECF2111CFCF0AC0BA
:1017100080919B03882361F0853061F08091E8001F
:1017200083FD0AC08091E80082FFF2CF80E0089537
:1017300082E0089583E0089581E008952091A20356
:101740003091A3032617370748F06115710539F466
:101750002091E8002E772093E80001C0B901FC0138
:1017600020E06115710591F180919B03882309F4B4
:1017700040C0853009F43FC08091E80083FD3DC042
:101780008091E80082FD2FC08091E80080FFE9CFC2
:101790002091F3008091F20090E0922B6115710589
:1017A00059F08830910540F424912093F10031964E
:1017B000615071090196F2CF21E0089709F020E00D
:1017C0008091E8008E778093E800CBCF2111CCCFB9
:1017D0000AC080919B03882361F0853061F080917D
:1017E000E80083FD0AC08091E80082FFF2CF80E02C
:1017F000089582E0089583E0089581E00895982F88
:10180000973068F59093E900981739F07091EC00E3
:101810002091ED005091F00003C0242F762F50E06E
:1018200021FD02C09F5FECCF3091EB003E7F3093F3
:10183000EB003091ED003D7F3093ED003091EB00F7
:1018400031603093EB007093EC002093ED005093E7
:10185000F0002091EE0027FDE5CF80E008958F7025
:101860008093E90081E0089580919C0387FF11C077
:101870008091E80082FD05C080919B038111F8CF23
:1018800011C08091E8008B770BC080919B03882367
:1018900049F08091E80080FFF8CF8091E8008E77D2
:1018A0008093E80008952091E4003091E50095E6EA
:1018B0004091EC00842F817040FF23C08091E800AC
:1018C00080FD1DC080919B03882399F0853099F09D
:1018D0008091EB0085FD11C04091E4005091E5003E
:1018E0002417350729F3915011F09A01E1CF84E0D4
:1018F000089582E0089583E0089581E0089580E0EE
:1019000008954091E80042FFDDCF08950E94F40C55
:101910000E94FC0CE0EEF0E0808181608083E8EDC5
:10192000F0E080818F77808319BCA7EDB0E08C91C7
:101930008E7F8C9380818F7E808310929A0308958E
:101940000F931F93CF93DF930E94F40C0E94FC0C23
:10195000C8EDD0E088818F7788838881806888830C
:1019600088818F7D888319BC10929B031092970306
:10197000109299031092980300EE10E0F801808114
:101980008B7F808388818160888342E060E080E093
:101990000E94FF0BE1EEF0E080818E7F8083E2EE1B
:1019A000F0E0808181608083808188608083F8019D
:1019B00080818E7F8083888180618883DF91CF9151
:1019C0001F910F910895E8EDF0E080818F7E808374
:1019D000E7EDF0E080818160808384E082BF81E078
:1019E00080939A030C94A00CE8EDF0E080818E7F48
:1019F00080831092E20008951092DA001092E100C4
:101A000008951F920F920FB60F9211242F933F93B8
:101A10004F935F936F937F938F939F93AF93BF93F6
:101A2000EF93FF938091E10082FF0BC08091E20071
:101A300082FF07C08091E1008B7F8093E1000E94CC
:101A4000D6088091DA0080FF1FC08091D80080FF07
:101A50001BC08091DA008E7F8093DA008091D900DC
:101A600080FF0DC080E189BD82E189BD09B400FE1F
:101A7000FDCF81E080939B030E94C40805C019BC80
:101A800010929B030E94D2088091E10080FF19C050
:101A90008091E20080FF15C08091E2008E7F8093EC
:101AA000E2008091E20080618093E2008091D800A2
:101AB00080628093D80019BC85E080939B030E94CC
:101AC000AC098091E10084FF30C08091E20084FF86
:101AD0002CC080E189BD82E189BD09B400FEFDCF43
:101AE0008091D8008F7D8093D8008091E1008F7E17
:101AF0008093E1008091E2008F7E8093E2008091EC
:101B0000E20081608093E20080919703882311F0C6
:101B100084E007C08091E30087FD02C081E001C03E
:101B200083E080939B030E94C1098091E10083FFC1
:101B300029C08091E20083FF25C08091E100877F6A
:101B40008093E10082E080939B0310929703809141
:101B5000E1008E7F8093E1008091E2008E7F809390
:101B6000E2008091E20080618093E20042E060E068
:101B700080E00E94FF0B8091F00088608093F0006D
:101B80000E94D508FF91EF91BF91AF919F918F91E6
:101B90007F916F915F914F913F912F910F900FBE69
:101BA0000F901F9018951F920F920FB60F9211244D
:101BB0002F933F934F935F936F937F938F939F9355
:101BC000AF93BF93CF93DF93EF93FF93C091E9005F
:101BD000CF708091EC00D82FD17080FDD0E81092AA
:101BE000E9008091F000877F8093F00078940E9454
:101BF000170E1092E9008091F00088608093F00049
:101C0000CD2BCF70C093E900FF91EF91DF91CF9181
:101C1000BF91AF919F918F917F916F915F914F9104
:101C20003F912F910F900FBE0F901F9018951F930B
:101C3000CF93DF93CDB7DEB7AA970FB6F894DEBF88
:101C40000FBECDBFECE9F3E08091F100819323E07A
:101C5000E43AF207C9F70E94F0088091E80083FF98
:101C600024C180919C0390919D03492F50E04A30FC
:101C7000510508F01AC1FA01EA5AFF4F0C94D22517
:101C8000803881F0823809F010C18091A0038F70F4
:101C90008093E9008091EB0085FB882780F9109202
:101CA000E90006C080919803909199039111826098
:101CB0009091E800977F9093E8008093F100109254
:101CC000F100C8C0282F2D7F09F0EFC0882319F03C
:101CD000823061F0EAC080919E03813009F0E5C056
:101CE000933009F080E0809399032BC080919E038C
:101CF000811127C08091A0038F7009F4D6C0809312
:101D0000E9002091EB0020FF1CC0933021F480916A
:101D1000EB00806214C09091EB0090619093EB0017
:101D200021E030E0A90102C0440F551F8A95E2F777
:101D30004093EA001092EA008091EB008860809363
:101D4000EB001092E9008091E800877F86C0811146
:101D5000ACC010919E031F778091E3008078812BA7
:101D60008093E3008091E800877F8093E8000E94E1
:101D7000340C8091E80080FFFCCF8091E300806804
:101D80008093E300111102C082E001C083E08093E0
:101D90009B038BC08058823008F087C080919E03DF
:101DA00090919F038C3D53E0950779F583E08A83FA
:101DB0008AE289834FB7F894DE01139620E03EE073
:101DC00051E2E32FF0E050935700E49120FF03C06D
:101DD000E295EF703F5FEF708E2F90E0EA3010F0E9
:101DE000C79601C0C0968D939D932F5F243149F70C
:101DF0004FBF8091E800877F8093E8006AE270E03F
:101E0000CE0101960E94400B14C0AE014F5F5F4FA0
:101E10006091A0030E94890ABC01892B09F445C086
:101E20009091E800977F9093E80089819A810E94C1
:101E30009E0B8091E8008B778093E80036C0803855
:101E4000A1F58091E800877F8093E8008091970357
:101E50008093F1008091E8008E778093E8000E94E3
:101E6000340C23C0811121C080919E0390919F0367
:101E700099270297D4F48091E800877F8093E80047
:101E800080919E03809397030E94340C8091970366
:101E9000811106C08091E30087FD02C081E001C08E
:101EA00084E080939B030E94D7088091E80083FF21
:101EB0000AC08091E800877F8093E8008091EB0062
:101EC00080628093EB00AA960FB6F894DEBF0FBE37
:101ED000CDBFDF91CF911F91089590938F02809392
:101EE0008E020895E0918E02F0918F02309721F0DA
:101EF0000190F081E02D099480E00895EF92FF9227
:101F00000F931F93CF93DF93E0918E02F0918F0296
:101F10003097B1F18C010280F381E02D0995809119
:101F2000860382FF2DC080FF04C08CEB93E00E94EB
:101F30009A05E80110E286EBE82E83E0F82E809106
:101F4000860380FF0BC088811F928F93FF92EF92D0
:101F50000E9433060F900F900F900F901150219612
:101F60001111EDCF8091860380FF0AC084EB93E0CE
:101F7000DF91CF911F910F91FF90EF900C949A05F4
:101F8000DF91CF911F910F91FF90EF900895E09115
:101F90008E02F0918F02309721F00480F581E02DC0
:101FA00009940895CF93DF9320918C0230918D0294
:101FB0002817390709F190938D0280938C02E091E4
:101FC0008E02F0918F023097B9F0EC010680F78114
:101FD000E02D09958091860382FF0EC080FF0CC022
:101FE000DF93CF9386EA93E09F938F930E9433060B
:101FF0000F900F900F900F90DF91CF910895CF9396
:10200000DF9320918A0230918B022817390709F15A
:1020100090938B0280938A02E0918E02F0918F025E
:102020003097B9F0EC010084F185E02D099580919D
:10203000860382FF0EC080FF0CC0DF93CF9386E93A
:1020400093E09F938F930E9433060F900F900F9011
:102050000F90DF91CF9108950C94EE100E94271DF0
:102060000C943C068F929F92AF92BF92CF92DF92D8
:10207000EF92FF920F931F93CF93DF9300D000D086
:102080001F92CDB7DEB70E946B0601E912E0F12C7A
:102090008F2D0E9432074C01F801A080B180A82644
:1020A000B926A114B10439F4F3940E5F1F4FF8E080
:1020B000FF12EECF39C08091860381FD0E94EF10A0
:1020C000E12CCC24C394D12CC5018C219D21892BDA
:1020D00021F1E982FA8221E0C4018C219D21892B22
:1020E00009F420E02B830E94301D8160782F9D83AE
:1020F0008C8349815A816B818D810E942511498190
:102100005A816B817C818D810E94A71CF80180819E
:1021100091818C259D2591838083E394CC0CDD1CDB
:10212000F0E1EF12D1CFC0CF8FEF89838A831B827A
:102130000E94301D8160782F9D838C8349815A8154
:102140006B818D810E9425110E94A61C0E94EE1FAA
:102150000E94720F90919002891759F10E94720F9C
:10216000809390029091860392FF0EC090FF0CC066
:102170001F928F9387EC93E09F938F930E94330677
:102180000F900F900F900F90809190020F900F90F2
:102190000F900F900F90DF91CF911F910F91FF90B3
:1021A000EF90DF90CF90BF90AF909F908F900C9466
:1021B000B81C0F900F900F900F900F90DF91CF9160
:1021C0001F910F91FF90EF90DF90CF90BF90AF9055
:1021D0009F908F9008950C943F0708950895EF9273
:1021E000FF920F931F93CF93DF9381EE93E00E94B2
:1021F0009A05C0E0D0E082E3E82E81E0F82E02EDFF
:1022000013E08C2F0E9432070E94931CFF92EF92E2
:102210009F938F93DF93CF931F930F930E94330667
:1022200021968DB79EB708960FB6F8949EBF0FBE45
:102230008DBFC830D10529F7DF91CF911F910F9144
:10224000FF90EF90089508950895CF93DF93CDB751
:10225000DEB72B970FB6F894DEBF0FBECDBF942F1D
:102260004F83252F588769877A878B874A855B85B7
:10227000452B31F02F3F31F481E09F3F19F403C02B
:1022800081E001C080E080FD07C04F8158856985ED
:102290007A858B850E94A71CDE01119686E0FD01E0
:1022A00011928A95E9F785E0FE01379601900D922B
:1022B0008A95E1F749815A816B817C818D819E816C
:1022C0000E9456182B960FB6F894DEBF0FBECDBFF6
:1022D000DF91CF910895CF93882309F465C0C82F6B
:1022E0008CEF8C0F813A20F080E58C0F8E3248F411
:1022F0008C2F0E943823811157C08C2F0E943E1BC7
:102300000CC080E28C0F883058F4C77081E001C0A7
:10231000880FCA95EAF70E94E31BCF910C94271C03
:102320008BE58C0F833078F4C53A29F0C63A31F04A
:1023300083E890E005C081E890E002C082E890E088
:10234000CF910C94D20F88E58C0F853168F5C83A8F
:1023500089F0C93A91F0CA3A99F0CB3AA1F0CC3A57
:10236000A9F0CD3AB1F0CE3AB9F0CF3AC1F080E061
:1023700090E017C082EE90E014C089EE90E011C0AA
:102380008AEE90E00EC085EB90E00BC086EB90E00B
:1023900008C083EB90E005C084EB90E002C087EBBF
:1023A00090E0CF910C94FF0FCF910895882349F1CD
:1023B0009CEF980F913A20F090E5980F9E3218F418
:1023C0000E948E1B0DC090E2980F983058F48770D1
:1023D00091E001C0990F8A95EAF7892F0E94E91BC5
:1023E0000C94271C9BE5980F933020F480E090E03C
:1023F0000C94D20F885A853120F480E090E00C9440
:10240000FF0F0895882321F00E94E31B0C94271CE2
:102410000895882321F00E94E91B0C94271C08953D
:102420000E94031C0E94D21B0E94271C0E94932022
:102430000E94611F80E090E00E94D20F80E090E057
:102440000C94FF0F0E94F31B0C941012CF92DF929A
:10245000EF92FF920F931F93CF93DF9300D000D0A2
:102460001F92CDB7DEB76C010E94BA1C811101C367
:1024700085E0F601DE01119601900D928A95E1F753
:10248000F60140815181238134812115310531F0DC
:102490005F3F31F481E04F3F19F403C081E001C098
:1024A00080E080FDE6C2F601F280E580E2948FE0F4
:1024B000E82249835A83FB82722F3D832C836F2D40
:1024C0008D810E94BA1A8C010E94B91A0E94A91922
:1024D000E12FE295EF708E2F90E0FC01E05AFF4F64
:1024E0000C94D225812F807F1F70882311F01295C4
:1024F000107FFF2049F0112309F452C2812F0E945E
:10250000F61B0E94271C4CC2802F0E94D61111235B
:1025100009F4AFC2812F0E94FC1B0F900F900F9007
:102520000F900F90DF91CF911F910F91FF90EF903F
:10253000DF90CF900C94271C812F807F1F708032FA
:1025400011F01295107F002319F0013009F12BC012
:10255000FF20A9F0EE2059F1F1E0812FEF1228C001
:102560000F900F900F900F900F90DF91CF911F91D0
:102570000F91FF90EF90DF90CF900C94061CEE200F
:1025800021F021E0E21609F474C20E940F1C2DC054
:10259000FF20E9F085E08E1508F46BC20E94E01B75
:1025A000812329F022C0FF20F1F0E11015C0812F16
:1025B0000F900F900F900F900F90DF91CF911F9180
:1025C0000F91FF90EF90DF90CF900C94021294E067
:1025D0009E1508F44EC209C0F601858180FFE0C156
:1025E0008F708583E4CFE110EEC1812F61C1812F0F
:1025F00086958695837019F08130B9F03AC2FF2034
:1026000019F0C801937002C080E090E00F900F9025
:102610000F900F900F90DF91CF911F910F91FF902E
:10262000EF90DF90CF900C94D20FFF2019F0C801EB
:10263000937002C080E090E00F900F900F900F9089
:102640000F90DF91CF911F910F91FF90EF90DF904E
:10265000CF900C94FF0F802FFF2019F00E94741E62
:1026600002C00E94DC1E0F900F900F900F900F90F1
:10267000DF91CF911F910F91FF90EF90DF90CF905E
:102680000C94611F812F837009F070C0F110F1C1AB
:10269000202F229526952770220F220F602F6F7012
:1026A000862F90E0A0E0B0E06C017D01022E04C016
:1026B000CC0CDD1CEE1CFF1C0A94D2F704FF12C0E8
:1026C0008FE090E0A0E0B0E004C0880F991FAA1F3F
:1026D000BB1F2A95D2F7BC01CD01609570958095FE
:1026E000909503C060E070E0CB01169516951370CD
:1026F0001230B1F040F56C297D298E299F291130C7
:1027000031F10F900F900F900F900F90DF91CF91BC
:102710001F910F91FF90EF90DF90CF900C94CE1906
:102720006C297D298E299F290F900F900F900F9073
:102730000F90DF91CF911F910F91FF90EF90DF905D
:10274000CF900C94E8190E94CE19C701B6010F90E2
:102750000F900F900F900F90DF91CF911F910F91DD
:10276000FF90EF90DF90CF900C94B419FF2019F0F8
:10277000812F817001C08695882309F47AC1202FAA
:10278000229526952770220F220F602F6F70862FBB
:1027900090E0A0E0B0E06C017D01022E04C0CC0C02
:1027A000DD1CEE1CFF1C0A94D2F704FF12C08FE060
:1027B00090E0A0E0B0E004C0880F991FAA1FBB1FE3
:1027C0002A95D2F7BC01CD016095709580959095C2
:1027D00003C060E070E0CB011695169513701230BF
:1027E000B1F040F56C297D298E299F29113031F1F6
:1027F0000F900F900F900F900F90DF91CF911F913E
:102800000F91FF90EF90DF90CF900C94951A6C2968
:102810007D298E299F290F900F900F900F900F9078
:10282000DF91CF911F910F91FF90EF90DF90CF90AC
:102830000C94A71A0E94951AC701B6010F900F9029
:102840000F900F900F90DF91CF911F910F91FF90FC
:10285000EF90DF90CF900C94831A003FC1F128F4E1
:1028600080E4800F803250F096C0023F09F45EC0D1
:1028700008F449C0033F09F46CC08DC0F02FF0711B
:10288000EF2E812F8F71FF2051F00E941C1A802F94
:10289000EE2019F08295807F8BCE8F7089CE0E94BA
:1028A0003D1A802FEE2019F08295807F01C08F7035
:1028B0000F900F900F900F900F90DF91CF911F917D
:1028C0000F91FF90EF90DF90CF900C940912FF20B2
:1028D000A9F024E02E1508F4CCC0812F8F710F9041
:1028E0000F900F900F900F90DF91CF911F910F914C
:1028F000FF90EF90DF90CF900C94621A85E08E15D8
:1029000008F4B7C0EACFFF2099F0812F8F710F90A4
:102910000F900F900F900F90DF91CF911F910F911B
:10292000FF90EF90DF90CF900C941C1AFF2069F37A
:10293000812F8F710F900F900F900F900F90DF915C
:10294000CF911F910F91FF90EF90DF90CF900C945B
:102950003D1AFF2089F0812F8F710F900F900F90FB
:102960000F900F90DF91CF911F910F91FF90EF90FB
:10297000DF90CF900C94071A0F900F900F900F904C
:102980000F90DF91CF911F910F91FF90EF90DF900B
:10299000CF900C94021AFF2099F0EE2009F4B5CFE5
:1029A000802F0F900F900F900F900F90DF91CF918D
:1029B0001F910F91FF90EF90DF90CF900C946B11CF
:1029C000EE2009F4B5CF802F0F900F900F900F904D
:1029D0000F90DF91CF911F910F91FF90EF90DF90BB
:1029E000CF900C94D611412F4F70602FC6010E94DA
:1029F000EE1D0F900F900F900F900F90DF91CF91E1
:102A00001F910F91FF90EF90DF90CF900C940419DD
:102A100001112FC0FF2069F10E9422129FEFE0E711
:102A2000F2E09150E040F040E1F700C000000F906C
:102A30000F900F900F900F90DF91CF911F910F91FA
:102A4000FF90EF90DF90CF900C94971D412F4F7027
:102A5000602FC6010F900F900F900F900F90DF9195
:102A6000CF911F910F91FF90EF90DF90CF900C943A
:102A7000F11D0F900F900F900F900F90DF91CF915D
:102A80001F910F91FF90EF90DF90CF9008951F93CB
:102A9000CF93DF9300D000D01F92CDB7DEB7942F35
:102AA0004983252F5A836B837C838D834C815D8181
:102AB000452B31F02F3F31F481E09F3F19F403C0E3
:102AC00081E001C080E0182F117080FD31C0498184
:102AD0005A816B817C818D810E94BA1A292F22959F
:102AE0002F702C3030F42A30A0F42250223030F0F5
:102AF00022C02C30C9F02F30B9F01DC0853A28F41F
:102B00008430C0F4823028F415C090E2980F9830D9
:102B100088F0883E30F4803E68F48450813A58F45E
:102B200009C0803F41F406C093FB112710F903C090
:102B300010E001C011E0812F0F900F900F900F90C7
:102B40000F90DF91CF911F910895CF93DF9300D025
:102B500000D01F92CDB7DEB70F900F900F900F905F
:102B60000F90DF91CF910895CF93DF9300D000D0E5
:102B700000D0CDB7DEB726960FB6F894DEBF0FBEF5
:102B8000CDBFDF91CF9108951F93CF93DF93C09175
:102B9000A10216E08091A202C81799F0D0E01C9F14
:102BA000F0011D9FF00D1124ED55FD4F4081518125
:102BB00062817381848195810E94B4152196C770CA
:102BC000E9CFDF91CF911F9108954091D3025091A9
:102BD000D4026091D5027091D6028091D702909173
:102BE000D8020C94B415CF938091D80282958F703F
:102BF00009F05FC08091D502882309F45AC0809102
:102C0000A102B091A2027091D302A091D40240918E
:102C1000D6025091D70291E07F3F09F090E0692FF2
:102C2000C6E08B1709F445C04115510521F0AF3FAF
:102C300021F020E003C021E001C0262F90E020FD1C
:102C400035C0C89FF001C99FF00D1124ED55FD4F0F
:102C500021812A132BC02081271328C02281211112
:102C600025C0238134812417350710F42150310900
:102C7000241B350B2C323140C8F42091D8022F7020
:102C800020612093D80226E0289FF001299FF00DB3
:102C90001124E855FD4F80818F708061808383ED22
:102CA00092E00E942612CF910C94C4150196877071
:102CB000B8CFCF910895AF92BF92CF92DF92EF92AB
:102CC000FF920F931F93CF93DF93CDB7DEB761973A
:102CD0000FB6F894DEBF0FBECDBF7C0185E0F701D3
:102CE000DE011D9601900D928A95E1F7D7014C9176
:102CF00011965C9111971296DC90129713960D9194
:102D00001C9114973091D3026091D4028091D60225
:102D10009091D702009731F06F3F31F421E03F3FAF
:102D200019F403C021E001C020E0B22FB170BB2E26
:102D300020FD76C1A090D502AA2009F4D1C020912F
:102D4000D8020817190750F0F801E81BF90BCF015A
:102D5000CC24C3948C329140D0F009C080959095DA
:102D6000800F911FCC24C3948C32914080F0C12CF1
:102D7000207F09F0A1C0702F198B088B6D2D8989D8
:102D80000E94A51583ED92E00E942612BDC0822FFD
:102D9000807F09F056C0561315C0431313C0CD2CC5
:102DA000D11010C02F7020612093D8020E94E51529
:102DB00083ED92E00E9426128091D802D7011596E9
:102DC0008C9362C10115110531F05F3F31F481E050
:102DD0004F3F19F403C081E001C080E080FD03C0D3
:102DE00081E08D2502C080E090E0B82FB170CB2E3D
:102DF00080FF1CC08091A1022091A20236E08217C0
:102E000009F41FC190E0389FF001399FF00D1124A3
:102E1000ED55FD4F6181561306C06081461303C016
:102E20006281D61203C001968770E9CFCD2CDD20D8
:102E300009F42AC18091D80281608093D802C12C04
:102E400023C1561308C0431306C0D11004C080919B
:102E5000D802D701B9C04D875E87DF86702F198BE6
:102E6000088B6D2D89890E944715882399F1DD20F3
:102E700089F12091D802822F82958F7090E002977D
:102E800074F08091D3029091D40298878F83198631
:102E90001B870A872C87CE0107960E94261286E0A0
:102EA000F701A3EDB2E001900D928A95E1F70E943F
:102EB000F3150E94E51511C0561781F14D875E8705
:102EC000DF86702F198B088B6D2D89890E9447151D
:102ED000811138C0C7010E942612CC24C394D4C0EB
:102EE0000817190708F446C0F801E81BF90BCF01D1
:102EF0008C32914008F446C0C12C702F198B088B7E
:102F00006D2D89890E94A515E3EDF2E086E0DF01D1
:102F10001D928A95E9F70E94E515B6C04313CECFFE
:102F2000D110CCCF8091D802F7018583C7010E94D0
:102F3000261286E0E3EDF2E0DF011D928A95E9F7C3
:102F4000CA2CA2C0DD2031F22091D802822F8295B6
:102F50008F7090E002970CF4A2CF8091D3029091F1
:102F6000D4029A8389831B821D830C832E83CE0116
:102F7000019693CF80959095800F911F8C32914050
:102F800008F0BACFCD2CDD2009F4A4CF561333C0FE
:102F9000431331C02091D80220FD24C0822F829596
:102FA0008F70482F50E041155105E1F0D70115967B
:102FB0002C9315974F30510549F08F5F982F9295BC
:102FC000907F822F8F70892B15968C93C7010E945A
:102FD000261286E0F701A3EDB2E001900D928A95EA
:102FE000E1F799CF86E0F701A3EDB2E001900D92F1
:102FF0008A95E1F749C04D875E87DF86702F198B70
:10300000088B6D2D89890E944715811148CF8091C9
:10301000D80281608093D802C7010E94261234C072
:10302000DD2009F457CF4D875E87DF86702F198B1F
:10303000088B6D2D89890E944715882309F44ACF92
:103040002ECF702F198B088B6D2D89890E94BA1A8B
:10305000292F22952F70223028F49F7039F081118A
:1030600005C00BC0243028F49F7049F4805E88307E
:1030700020F0C7010E942612BC2CCB2C05C0F70102
:103080009581907F99F7F9CF8C2D61960FB6F894C2
:10309000DEBF0FBECDBFDF91CF911F910F91FF908B
:1030A000EF90DF90CF90BF90AF9008951F93CF9394
:1030B000DF93CDB7DEB72C970FB6F894DEBF0FBE07
:1030C000CDBF4F83588769877A878B879C87CE01CE
:1030D00007960E945B168823D1F09F8188852A85F8
:1030E0003B85232B31F08F3F31F481E09F3F19F472
:1030F00003C081E001C080E080FD47C04F8158855A
:1031000069857A858B859C850E94B4153EC086E0D2
:10311000FE013796DE01119601900D928A95E1F736
:10312000FF81E8856A857B856115710531F0EF3F88
:1031300031F481E0FF3F19F403C081E001C080E079
:1031400080FD23C02091A20230E0C9010196877062
:1031500099274091A10250E084179507F1F1F98376
:10316000EA837D836C8396E0929FD001939FB00D9C
:103170001124AD55BD4FFE01319601900D929A95E7
:10318000E1F78093A2020E94C41516E08091A1028B
:103190009091A202891771F1189FC00111248D55D9
:1031A0009D4F0E945B16882329F1E091A1021E9F8A
:1031B000F0011124ED55FD4F4081518162817381F1
:1031C000848195810E94B4158091A10290E00196BE
:1031D000877099278093A102D9CF0E942212109262
:1031E000A2021092A102E3EDF2E086E0DF011D925F
:1031F0008A95E9F72C960FB6F894DEBF0FBECDBFC7
:10320000DF91CF911F910895DF92EF92FF920F937C
:103210001F93CF93DF93FC01892B09F488C0E12C25
:10322000F12CDD24D394EF0121968491853709F4A4
:1032300060C058F4843708F04EC0843008F068C08D
:103240008130D1F0823071F172C0883709F45BC0EF
:1032500050F4863709F453C0873709F068C08E2DC3
:103260000E94F01B52C09CE7980F903708F05FC097
:103270008F770E94D6114EC08F010E5F1F4FFE0147
:10328000849190E2980F983050F48770FD2D01C022
:10329000FF0F8A95EAF78F2F0E94F61B15C00E9438
:1032A0006B1114C08F010E5F1F4FFE01849190E2DD
:1032B000980F983068F48770FD2D01C0FF0F8A9534
:1032C000EAF78F2F0E94FC1B0E94271CE80122C0F6
:1032D0000E94D611FBCFCF010296FE01C491CC23F0
:1032E00061F0EFE9FFE03197F1F700C00000C15055
:1032F000F6CFCF010296FE01F490EC010BC00E94C4
:10330000E01BE82E07C00E94F31B0E94271C02C08E
:103310000E946B118F2D882341F0EFE9FFE0319778
:10332000F1F700C000008150F6CFFE017CCFDF91A5
:10333000CF911F910F91FF90EF90DF9008956093D0
:10334000590370935A0380935B0390935C030C942E
:10335000B71C089560935D0370935E0380935F03D1
:10336000909360030C94B61C0F931F9300915D0320
:1033700010915E0320915F0330916003602B712BED
:10338000822B932B60935D0370935E0380935F03A6
:10339000909360031F910F910C94B61C0F931F9391
:1033A00000915D0310915E0320915F0330916003F3
:1033B000602371238223932360935D0370935E03E4
:1033C00080935F03909360031F910F910C94B61C40
:1033D0000F931F9300915D0310915E0320915F0393
:1033E00030916003602771278227932760935D03E4
:1033F00070935E0380935F03909360031F910F911E
:103400000C94B61C60E070E0CB010C949F190F93F4
:103410001F9341E050E060E070E08A019B0104C02E
:10342000000F111F221F331F8A95D2F7C901B8015F
:103430001F910F910C949F190F931F9341E050E03F
:1034400060E070E004C0440F551F661F771F8A9527
:10345000D2F78091590390915A03A0915B03B091E8
:103460005C038A019B01082B192B2A2B3B2BC901DA
:10347000B8011F910F910C949F190F931F9341E076
:1034800050E060E070E004C0440F551F661F771FD6
:103490008A95D2F740955095609570958091590323
:1034A00090915A03A0915B03B0915C038A019B0148
:1034B000082319232A233B23C901B8011F910F9127
:1034C0000C949F190F931F9341E050E060E070E06F
:1034D00004C0440F551F661F771F8A95D2F780914D
:1034E000590390915A03A0915B03B0915C038A0148
:1034F0009B01082719272A273B27C901B8011F91DB
:103500000F910C949F190F931F93009159031091E1
:103510005A0320915B0330915C03602B712B822B4B
:10352000932B1F910F910C949F190F931F93009150
:10353000590310915A0320915B0330915C0360237F
:103540007123822393231F910F910C949F190F9342
:103550001F930091590310915A0320915B033091FE
:103560005C0360277127822793271F910F910C948A
:103570009F1908958F929F92AF92BF92DF92EF9220
:10358000FF920F931F93CF93DF9300D000D01F9231
:10359000CDB7DEB76B837C838D838A018C819D815F
:1035A000892B31F01F3F31F481E04F3F19F403C004
:1035B00081E001C080E080FF03C080E090E04DC06A
:1035C0008B818823D1F18090590390905A03A09069
:1035D0005B03B0905C0380915D0390915E03A091CA
:1035E0005F03B0916003882A992AAA2ABB2A8FE137
:1035F000E82EF12CD501C4010E2C04C0B695A79578
:10360000979587950A94D2F780FD06C081E0E81A65
:10361000F10880F7D12C07C0DE2CB8018E2D0E9456
:10362000C51D019799F380E1189FF0011124E7521D
:10363000FD4FE00FF11DD08209C080E1189FF0011D
:103640001124E752FD4FE00FF11DD08009831A834A
:1036500069817A818D2D0E94C51D0F900F900F906A
:103660000F900F90DF91CF911F910F91FF90EF90EE
:10367000DF90BF90AF909F908F90089590910F0131
:10368000992379F190911001992359F1982F9695EA
:10369000969596959F31A1F0E0911101F09112015C
:1036A000E90FF11D877021E030E0A90102C0440F4D
:1036B000551F8A95E2F7CA019181892B818308956C
:1036C0009091860390FF29C01F928F9385E194E02B
:1036D0009F938F930E9433060F900F900F900F903F
:1036E00008952091110130911201F90132969FEF56
:1036F00040E05191851789F09F3F19F4511101C0A5
:10370000942F4F5F4E31A9F79F3F39F0F901E90F30
:10371000F11D97FDFA9582830895089590910F0108
:10372000992381F190911001992361F1982F969539
:10373000969596959F31A9F0E0911101F0911201B3
:10374000E90FF11D877021E030E0A90102C0440FAC
:10375000551F8A95E2F7CA0180959181892381835B
:1037600008959091860390FF1CC01F928F9387EF5E
:1037700093E09F938F930E9433060F900F900F90CA
:103780000F900895E0911101F09112019F01225EC6
:103790003F4F9281891301C012823196E217F307DD
:1037A000C1F7089581E090E0E0911101F0911201DC
:1037B000E80FF91F1082019680329105A9F708954C
:1037C00080918503089590918503892B80938503CB
:1037D00008958095909185038923809385030895AA
:1037E0008093850308951092850308959091840332
:1037F000892B809384030895809590918403892375
:103800008093840308951092840308958093630342
:103810000E94301D9093620380936103089510927B
:103820006303109262031092610308958091110165
:1038300090911201FC0131969C01205E3F4F80E087
:10384000919191118F5FE217F307D1F70895E091FD
:103850001101F0911201809185038083E0911101A3
:10386000F0911201908180918403892B8083809153
:1038700063038823D9F10E94301D209161033091A8
:1038800062038217930748F00E94301D2091610364
:1038900030916203821B930B0AC00E94301D20915D
:1038A00061033091620320953095820F931F8C3213
:1038B000914070F08091860380FF08C083E394E01C
:1038C0009F938F930E9433060F900F900E940F1CBE
:1038D000E0911101F0911201908180916303892B95
:1038E00080830E94161C81110E940F1C809111017F
:1038F000909112010C947E0F90933F0180933E01B2
:1039000008958295982F937344E0949F9001112419
:103910008C7C86958695282B822F8575880F2A7A30
:103920002695822B0895CF93DF93D92F0E94811C77
:10393000C82F8D2F0E94811C2C2F30E0322F222780
:10394000A901482BCA01DF91CF9108950895CF9323
:10395000DF9300D000D01F92CDB7DEB70F900F904D
:103960000F900F900F90DF91CF91089508950895D3
:103970000C94EB1080E0089580919B03843021F13A
:103980001092870320E488E190E00FB6F894A895A0
:10399000809360000FBE2093600083B7817F8460B6
:1039A00083BF83B7816083BF7894889583B78E7F08
:1039B00083BF0FB6F894A8958091600088618093CA
:1039C0006000109260000FBE0895CF930E942311F3
:1039D0000E946B060E942411C0E08C2F0E943207C7
:1039E000892B29F4CF5FC830C1F780E001C081E0A6
:1039F000CF9108950E94ED100C9422121F920F9205
:103A00000FB60F9211248F939F93AF93BF93809122
:103A10008703811113C08091880390918903A0913D
:103A20008A03B0918B034196A11DB11D8093880339
:103A300090938903A0938A03B0938B03BF91AF91B6
:103A40009F918F910F900FBE0F901F90189582E05D
:103A500084BD93E095BD9AEF97BD80936E00089565
:103A60002FB7F8948091880390918903A0918A03DD
:103A7000B0918B032FBF08952FB7F89460918803FE
:103A80007091890380918A0390918B032FBF0895D1
:103A9000CF92DF92EF92FF920F931F932FB7F8947C
:103AA000409188035091890360918A0370918B0340
:103AB0002FBF6A017B01EE24FF248C0120E030E05F
:103AC000C016D106E206F30610F4415051099A01DE
:103AD000281B390BC9011F910F91FF90EF90DF90C8
:103AE000CF9008951F920F920FB60F9211248F93CB
:103AF0009F93AF93BF938091880390918903A09186
:103B00008A03B0918B030196A11DB11D8093880398
:103B100090938903A0938A03B0938B03BF91AF91D5
:103B20009F918F910F900FBE0F901F9018950E943C
:103B3000860CF89487E797E7909301088093000834
:103B400087E090EBDC018093A4039093A503A093FE
:103B5000A603B093A7039CE088E10FB6F894A8955C
:103B6000809360000FBE90936000FFCFE82FF0E0DD
:103B700080E1989FE00DF11D1124E052FF4F9491D8
:103B8000892F8F7092959F700895CF93C82FCB0186
:103B90000E94B61DE92F90E040E1E49F90011124BE
:103BA000282B392B2038310519F480E090E014C01F
:103BB000E770F0E028E0C29FE00DF11D112424E041
:103BC000EE0FFF1F2A95E1F7E80FF91FEE0FFF1F19
:103BD000E050F84985919491CF91089580E090E06C
:103BE0000895089580918E0380FF0BC060911601A7
:103BF00085E0689FB0011124759567957595679567
:103C00002BC081FF09C06091160185E0689FB0015B
:103C100011247595679520C082FF07C06091160139
:103C200085E0689FB001112417C090918F039923FC
:103C3000D1F060911501961788F72091160185E063
:103C4000289F90011124929FA001939F500D112451
:103C500070E0CA010E94BE256038710540F461150C
:103C6000710519F406C065E070E0862F08958FE7AE
:103C7000089581E0089580918E0380FF08C06091CF
:103C8000140170E0759567957595679521C081FF62
:103C900006C06091140170E07595679519C082FFA8
:103CA00004C06091140170E010C090918F039923BB
:103CB00099F0609113019617A0F780911401899FE4
:103CC000C001112470E00E94BE256038710540F4E7
:103CD0006115710519F406C061E070E0862F089542
:103CE0008FE7089581E00895803F21F40E94F21D3E
:103CF000819504C0813F29F40E94F21D80939203B4
:103D00000895823F21F40E94F21D819504C0833FF3
:103D100029F40E94F21D809391030895893F19F4BC
:103D20000E943B1E05C08A3F31F40E943B1E8195D4
:103D30008093930308958B3F21F40E943B1E81954D
:103D400004C08C3F29F40E943B1E80939403089585
:103D5000843F21F480919003816017C0853F21F456
:103D600080919003826011C0863F21F4809190037E
:103D700084600BC0873F21F480919003886005C068
:103D8000883F31F48091900380618093900308957F
:103D90008D3F21F480918E0381600BC08E3F21F412
:103DA00080918E03826005C08F3F29F480918E033D
:103DB000846080938E030895803F39F4809192034C
:103DC00087FF6CC01092920369C0813F29F48091F3
:103DD00092031816BCF362C090919103823F29F4BC
:103DE00097FF5CC01092910359C0833F19F41916D4
:103DF000CCF354C0893F41F48091930318160CF022
:103E00004DC0109293034AC08A3F29F480919303D6
:103E100087FF44C0F6CF8B3F39F48091940387FF2E
:103E20003DC0109294033AC08C3F29F480919403D2
:103E30001816BCF333C0843F21F4809190038E7F29
:103E400017C0853F21F4809190038D7F11C0863F7C
:103E500021F4809190038B7F0BC0873F21F48091E8
:103E60009003877F05C0883F31F4809190038F7E57
:103E70008093900313C08D3F21F480918E038E7F39
:103E80000BC08E3F21F480918E038D7F05C08F3F44
:103E900029F480918E038B7F80938E038091910310
:103EA00081110EC08091920381110AC08091930309
:103EB000811106C080919403811102C010928F037A
:103EC00008958091860383FF7EC08CE694E00E9473
:103ED0009A05809190031F928F9387E694E09F93B9
:103EE0008F930E94330685E694E00E949A058091A4
:103EF0009103282F082E000C330B3F938F9382E6FB
:103F000094E09F938F930E94330680E694E00E9492
:103F10009A0580919203282F082E000C330B3F93B3
:103F20008F938DE594E09F938F930E9433068BE5EA
:103F300094E00E949A0580919303282F082E000C8C
:103F4000330B3F938F9388E594E09F938F930E9468
:103F5000330686E594E00E949A0580919403282F09
:103F6000082E000C330B3F938F9383E594E09F93CF
:103F70008F930E94330680E594E00E949A05809119
:103F80008F031F928F938DE494E09F938F930E94F1
:103F900033068BE494E00E949A0580918E031F9271
:103FA0008F9388E494E09F938F930E94330685E477
:103FB00094E00E949A058DB79EB74C960FB6F89480
:103FC0009EBF0FBE8DBF80E993E00E94C70F0E9485
:103FD000301D90938D0380938C0308951F93CF938E
:103FE000DF9380918C0390918D030E94481DAC015A
:103FF00090918F03992321F02091170130E006C0A2
:10400000209118018AE0289F90011124421753073C
:1040100008F485C080919103C0919203D0919303DD
:1040200010919403811107C0C11175C0D11173C0E3
:10403000111171C074C09F3F19F09F5F90938F035F
:10404000181624F40E94F21D80939103809191032D
:1040500087FF05C00E94F21D8195809391031C1675
:1040600024F40E94F21D809392038091920387FFB3
:1040700005C00E94F21D8195809392036091910387
:10408000662331F1C0919203CC2311F1062E000C6E
:10409000770B880B990B0E94C52423E333E343E39A
:1040A0005FE30E9429250E948D24609391036C2F69
:1040B000CC0F770B880B990B0E94C52423E333E3C5
:1040C00043E35FE30E9429250E948D2460939203BD
:1040D0001D1624F40E943B1E80939303809193034A
:1040E00087FF05C00E943B1E8195809393031116A4
:1040F00024F40E943B1E809394038091940387FFD5
:1041000005C00E943B1E819580939403DF91CF915F
:104110001F910C94611F9F3F09F08FCFA0CFDF91BB
:10412000CF911F910895E0E9F3E085E0DF011D9252
:104130008A95E9F710928F0310928E0308958FE805
:1041400096E00E949A051F9281E08F931F9285E06E
:104150008F9381E496E09F938F930E9433060F9094
:104160000F900F900F900F900F9008958330E9F10A
:1041700028F4813061F0823009F10895853009F426
:1041800062C008F449C0863009F474C00895809173
:104190001801262F30E0280F311D2F3F310524F460
:1041A000680F6093180103C08FEF8093180180910E
:1041B00018011F928F938AE795E072C080911701D2
:1041C000262F30E0280F311D2F3F310524F4680FD2
:1041D0006093170103C08FEF80931701809117013F
:1041E0001F928F9388E695E05BC080911601262F81
:1041F00030E0280F311D2F3F310524F4680F609304
:10420000160103C08FEF80931601809116011F9253
:104210008F9385E595E044C080911501262F30E00D
:10422000280F311D2F3F310524F4680F60931501CD
:1042300003C08FEF80931501809115011F928F931A
:1042400080E495E02DC080911401262F30E0280FE6
:10425000311D2F3F310524F4680F6093140103C012
:104260008FEF80931401809114011F928F9387E246
:1042700095E016C080911301262F30E0280F311DE4
:104280002F3F310524F4680F6093130103C08FEFB3
:1042900080931301809113011F928F938CE095E01E
:1042A0009F938F930E9433060F900F900F900F9063
:1042B0000895833081F128F4813059F08230D1F0B3
:1042C0000895853009F449C0B8F1863009F456C024
:1042D000089580911801681720F4861B80931801B7
:1042E00002C010921801809118011F928F938DEFD8
:1042F00094E054C080911701681720F4861B8093C6
:10430000170102C010921701809117011F928F931D
:104310008BEE94E043C080911601681720F4861B51
:104320008093160102C010921601809116011F920F
:104330008F9388ED94E032C080911501681720F4C6
:10434000861B8093150102C0109215018091150102
:104350001F928F9383EC94E021C080911401681721
:1043600020F4861B8093140102C0109214018091E6
:1043700014011F928F938AEA94E010C08091130178
:10438000681720F4861B8093130102C0109213015A
:10439000809113011F928F938FE894E09F938F93E6
:1043A0000E9433060F900F900F900F900895CF93B7
:1043B000C82F1F928F9384E997E09F938F930E9459
:1043C000330681E090E0A0E0B0E0BC01CD0104C084
:1043D000660F771F881F991FCA95D2F70E94AA19E6
:1043E0000F900F900F900F90CF910C942212CF93BB
:1043F0008732A8F58E3108F02BC1803109F49FC0B7
:10440000F8F4873009F464C0A8F4863009F024C1B8
:1044100080918603817F8E7F8093860389E997E070
:104420000E949A0583E89AE00E949A0581E08093B1
:1044300096034CC08B30F1F18E3009F46CC00CC186
:10444000863109F4B0C020F4813109F4EDC004C113
:10445000893109F491C08B3109F449C0FDC088331A
:1044600049F150F4893209F4F1C0853309F4EEC002
:10447000873209F0F1C0EAC0833409F4E7C028F4B8
:104480008A3308F4E9C08953E4C0883409F0E4C0F1
:104490000E94221282E79AE00E949A052FEF83ED94
:1044A00090E3215080409040E1F700C000000E945E
:1044B000971D0CC080EC97E05CC089E59AE00E94F3
:1044C0009A0580918603816080938603C1E0C9C00C
:1044D00080918603C82FC17080FFEFCF85E69AE0F8
:1044E0000E949A0580918603817F8E7F3DC09091C6
:1044F000860391FBCC27C0F981E0C827892FC0FB38
:1045000081F980938603CC2319F08CE49AE027C0CC
:104510008EE39AE02EC09091860392FBCC27C0F9DF
:1045200081E0C827892FC0FB82F980938603CC23C2
:1045300019F08FE29AE013C08FE19AE01AC09091CF
:10454000860393FBCC27C0F981E0C827892FC0FBE5
:1045500083F980938603CC2351F083E19AE00E9493
:104560009A05809186038160809386037AC086E0F5
:104570009AE00E949A05AACF87EF99E00E949A05D7
:104580008EEC99E00E949A058CE899E00E949A05C9
:1045900083E699E00E949A0589E199E00E949A05D4
:1045A0008EEE98E0E6CF80EE98E00E949A050E9499
:1045B000720F1F928F9386EC98E09F938F930E94C7
:1045C000330680910F011F928F938FEA98E09F939B
:1045D0008F930E943306809189021F928F938CE9FA
:1045E00098E09F938F930E943306809110011F9251
:1045F0008F9389E898E09F938F930E9433060E94DF
:104600003C1D9F938F937F936F9382E798E09F93D6
:104610008F930E9433068DB79EB746960FB6F894D7
:104620009EBF0FBE8DBF52CF0E942212C0911001BB
:1046300081E0C827C0931001CC2329F088E698E0D8
:104640000E949A050EC08DE598E093CF80E001C0EE
:104650008D510E94D7213ACF8BE598E00E949A05B0
:10466000C0E08C2FCF91089580E008950C943423FE
:10467000CF93C82F80919603813071F020F0823063
:1046800009F44BC042C1E0911101F0911201808107
:10469000823209F03CC107C0E0911101F091120192
:1046A0008081823261F48C2F0E943623811104C0F4
:1046B0008C2F0E94F7212FC081E090E02CC08C2F1E
:1046C0000E943423811126C0C431E1F070F4CB3054
:1046D00081F0C031D1F40E949F208CE897E00E94C5
:1046E0009A0582E08093960315C0C93259F0C83309
:1046F00061F489E997E00E949A0580E997E00E94B9
:104700009A0508C01092960304C18AE897E00E94B7
:104710009A05FFC081E08170FEC0C43228F5CE3119
:1047200008F0C1C0CB30A1F1D0F4C73009F0D3C03C
:104730008EE18093180182E3809317018AE08093D1
:10474000160184E18093150188E08093140188E2CA
:104750008093130180E396E00E949A05BFC0C331A5
:1047600049F1C431C1F0B7C0CB3409F4A9C028F471
:10477000C93289F0C83361F0AEC0C13509F49EC0BA
:10478000C23509F499C0CE3409F0A5C06AE09EC0D4
:104790000E949F20A3C080919503882319F0109256
:1047A00095039CC08DE396E00E949A0581E080937A
:1047B0009603B1C087E196E00E949A0585E096E0F5
:1047C0000E949A05809118011F928F9382E096E0D3
:1047D0009F938F930E94330680E096E00E949A0593
:1047E0008EEE95E00E949A05809117011F928F939B
:1047F0008BEE95E09F938F930E94330689EE95E0B0
:104800000E949A058AED95E00E949A058091160112
:104810001F928F9387ED95E09F938F930E943306AD
:1048200085ED95E00E949A0584EC95E00E949A053A
:10483000809115011F928F9381EC95E09F938F9348
:104840000E9433068FEB95E00E949A058AEA95E074
:104850000E949A05809114011F928F9387EA95E038
:104860009F938F930E94330685EA95E00E949A05F4
:104870008EE895E00E949A05809113011F928F9314
:104880008BE895E09F938F930E94330689E895E02B
:104890000E949A058DB79EB748960FB6F8949EBFB2
:1048A0000FBE8DBF1BC0CE51EC2FF0E0ED5CFE4F74
:1048B00080818093950312C061E003C061E006C06F
:1048C0006AE0809195030E94B62008C0809195030C
:1048D0000E94592103C08EE296E013C08091950397
:1048E000882369F01F928F9388E296E09F938F93BD
:1048F0000E9433060F900F900F900F9004C085E236
:1049000096E00E949A0581E006C01092960380E02E
:1049100002C080E000CFCF9108950E949424689453
:10492000B1110C94232508950E94082588F09F5703
:1049300098F0B92F9927B751B0F0E1F0660F771FC3
:10494000881F991F1AF0BA95C9F714C0B13091F0B9
:104950000E942225B1E008950C942225672F782F1C
:104960008827B85F39F0B93FCCF38695779567957E
:10497000B395D9F73EF490958095709561957F4FEA
:104980008F4F9F4F0895E89409C097FB3EF4909590
:104990008095709561957F4F8F4F9F4F9923A9F018
:1049A000F92F96E9BB279395F695879577956795A7
:1049B000B795F111F8CFFAF4BB0F11F460FF1BC0EB
:1049C0006F5F7F4F8F4F9F4F16C0882311F096E97E
:1049D00011C0772321F09EE8872F762F05C066232C
:1049E00071F096E8862F70E060E02AF09A95660FE5
:1049F000771F881FDAF7880F9695879597F908959E
:104A000057FD9058440F551F59F05F3F71F047957F
:104A1000880F97FB991F61F09F3F79F08795089564
:104A2000121613061406551FF2CF4695F1DF08C083
:104A3000161617061806991FF1CF869571056105A0
:104A400008940895E894BB2766277727CB0197F948
:104A500008950E943C250C94AD250E949F2538F0B6
:104A60000E94A62520F0952311F00C9496250C9415
:104A70009C2511240C9423250E94002570F3959FFA
:104A8000C1F3950F50E0551F629FF001729FBB2745
:104A9000F00DB11D639FAA27F00DB11DAA1F649FE1
:104AA0006627B00DA11D661F829F2227B00DA11D94
:104AB000621F739FB00DA11D621F839FA00D611D1A
:104AC000221F749F3327A00D611D231F849F600D3B
:104AD000211D822F762F6A2F11249F5750409AF064
:104AE000F1F088234AF0EE0FFF1FBB1F661F771FF0
:104AF000881F91505040A9F79E3F510580F00C94BB
:104B000096250C9423255F3FE4F3983ED4F38695D5
:104B100077956795B795F795E7959F5FC1F7FE2B5A
:104B2000880F911D9695879597F9089597F99F6736
:104B300080E870E060E008959FEF80EC0895002425
:104B40000A941616170618060906089500240A94F2
:104B500012161306140605060895092E0394000C78
:104B600011F4882352F0BB0F40F4BF2B11F460FF07
:104B700004C06F5F7F4F8F4F9F4F089597FB072EA5
:104B800016F4009407D077FD09D00E94D82507FCC1
:104B900005D03EF4909581959F4F0895709561954D
:104BA0007F4F0895EE0FFF1F0590F491E02D0994BB
:104BB000AA1BBB1B51E107C0AA1FBB1FA617B70743
:104BC00010F0A61BB70B881F991F5A95A9F780955F
:0C4BD0009095BC01CD010895F894FFCF32
:104BDC0068010000FF4F07DF07BC0786075207017B
:104BEC000164032808140A321E404D36223956033C
:104BFC000903D302B1027802EB0104021D02360252
:0E4C0C00560200010203040506070809000015
:106800000000000000000000040005000600070072
:10681000080009000A000B000C000D000E000F001C
:1068200010001100120013001400150016001700CC
:10683000180019001A001B001C001D001E001F007C
:10684000200021002200230024002500260027002C
:10685000280029002A002B002C002D002E002F00DC
:1068600030003100000033003400350036003700BE
:10687000380039003A003B003C003D003E003F003C
:106880004000410042004300440045000000000079
:106890000000490000004B004C0000004E004F007B
:1068A000500051005200530054005500560057004C
:1068B000580059005A005B005C005D005E005F00FC
:1068C0006000610062006300000000000000000042
:1068D00000000000000000000000000000000000B8
:1068E00000000000000000000000000000000000A8
:1068F000E000E100E200E300E400E500E600F1A1D1
:106900000000000000000000010001000100010083
:10691000010001000100010046000100010001002A
:1069200001000100470048000100010001000100D2
:10693000010001000100010001000100010001004F
:10694000010001000100010001000100010001003F
:10695000010001000100010001000100010001002F
:106960000100010000000100010001000100010020
:10697000010001000100010001000100010001000F
:106980000100010001000100010001000000000001
:106990000000010000004A00010000004D004D0011
:1069A0004A004E004B0001000100010001000100FF
:1069B00001000100010001000100010001000100CF
:1069C00001000100010001000000000000000000C3
:1069D00000000000000000000000000000000000B7
:1069E00000000000000000000000000000000000A7
:1069F000010001000100010065000100010001002B
:00000001FF
